:020000040000FA
:02000000FA28DC
:080008008C00030E8D008B1E1D
:100010000B280B1910280B1EF5288B18B028F52873
:100020001118152891186C2883280F08023C031812
:100030001A28652800300E02031D2128FF30860093
:100040005C2801300E02031D2828FD3086005C2844
:1000500002300E02031D2F28F93086005C28033081
:100060000E02031D3628F13086005C2804300E0293
:10007000031D3D28B13086005C2805300E02031DAB
:100080004428913086005C2806300E02031D4B2860
:10009000813086005C2807300E02031D5228013093
:1000A00086005C2808300E02031D5928FF308600A8
:1000B0005C28013086005C288E0A0E08093C031873
:1000C00063288E018F0A0B11F528FF3086000B166E
:1000D0008B128B100B11F52812187028121481281E
:1000E000910111150B128B100130940093008514AF
:1000F000831603138115011181100110831203135C
:1001000081280B11F52814081002031CA728930856
:10011000031D9528930A810183160313811501118C
:100120008110011083120313AC281308203C03181C
:10013000A528940A930181018316031381110115E7
:100140008110011483120313AC28930AAC280B16F8
:100150008B108B120B11F528023085060B11F52838
:10016000911CE62081019201900A1008063C0318B8
:10017000BC2801309000BC2801301002031DC328A8
:100180007F308600E22802301002031DCA28E730C3
:100190008600E22803301002031DD1286730860054
:1001A000E22804301002031DD828A5308600E2287A
:1001B00005301002031DDF2825308600E22881303B
:1001C0008600E228023085068B10F52891019114F3
:1001D0008B168101831603138111011581140114FB
:1001E000831203130B11920108000D0E83008C0E75
:1001F0000C0E090083120313850186018316031375
:10020000D53081001D308500013086008312031334
:100210008501FE3086008101A0308B008E018F01A8
:0C0220009001910111149201152915297B
:02400E00F33F7E
:00000001FF
